:0A0000000528000000000000912E0A
:10000A004D3083120313A2004830A3007A30A400B3
:10001A00A501A6012030A700A8012A30A900AA013B
:10002A00AB010230AC00AD014630AE005230AF0039
:10003A004530B0004530B100B2015030B3006F30E6
:10004A00B4007730B5006530B6007230B7002030A2
:10005A00B8003D30B9002030BA00BB014C30BC00BA
:10006A004F30BD004330BE004B30BF00C001C1015C
:10007A00C2010130CE000130CF006430D0007830A8
:10008A00D80007309F004530D10025246530D700BD
:10009A000C30EC00F6246330D2005030DA005527D9
:1000AA006830D3004C30DB0090308B046F30D400C2
:1000BA0003308316860466308312D5004C30DC0088
:1000CA00831605166C308312D60012109210C730B0
:1000DA0083169200DA272030D9000130E600013079
:1000EA00E7005130E800B6240B30FB002630FC0054
:1000FA005D30FD00FD0B7F28FC0B7F28FB0B7F2862
:10010A00000000000130EC00F624B7270330E000BD
:10011A009C2770088312DE004130FC00EE30FD009F
:10012A00FD0B9528FC0B952800005E08013A031D7B
:10013A009F28D5286430C500CB010130DE00093084
:10014A00E000E101B1264130FC00EE30FD00FD0B7C
:10015A00AC28FC0BAC28000001308312E0004508F3
:10016A00E100B1264130FC00EE30FD00FD0BBB285A
:10017A00FC0BBB28000002308312E0004B08E100B0
:10018A00B1264130FC00EE30FD00FD0BCA28FC0B05
:10019A00CA28000003308312E0005E08E100B1269D
:1001AA000330FB008A30FC005530FD00FD0BDB28D4
:1001BA00FC0BDB28FB0BDB2800000000013083125C
:1001CA00E0009C2770088312C5004130FC00EE3025
:1001DA00FD00FD0BEE28FC0BEE2800000230E000CB
:1001EA009C2770088312CB004130FC00EE30FD00E2
:1001FA00FD0BFD28FC0BFD2800000930E0009C27C0
:10020A0070088312C1004508E0004B08E100B722DC
:10021A008312D0035008003A031D87296430D000A6
:10022A001627C1308312E6004922E001E101D423F6
:10023A007008DD00D02683125D1F4C290130E600CC
:10024A000D30E7003C30E800B6244130FC00EE30C7
:10025A00FD00FD0B2E29FC0B2E2900004E08013A49
:10026A00031D4B29CE01DF015F084102031C4B2904
:10027A005F08E00011264130FC00EE30FD00FD0B66
:10028A004429FC0B44290000DF0A39295729013087
:10029A00E6000D30E7002E30E800B624E001112612
:1002AA000130CE0001304F06F0007008CF00700810
:1002BA00031967290230E6001030E7002930E80008
:1002CA00B6246E290230E6001030E7002730E80035
:1002DA00B624260803197D29A6010130E000450845
:1002EA00E100B12602308312E0004B08E100B1269A
:1002FA0083122D0803198729AD010930E00041084E
:10030A00E100B12605308312E0000430E1000A3032
:10031A00E200E301722570080319A529AC0A2C082A
:10032A00033A031D9929AC010530E0000430E100CD
:10033A000A30E200E301722570080319A5299929F8
:10034A002C08003A031DB82990308B040230E000D3
:10035A000130E1006B260130E6000130E700203071
:10036A00E800AA25DE292C08013A031DCB29903082
:10037A008B040130E0000130E1006B260230E60018
:10038A000130E7002030E800AA25DE292C08023ACD
:10039A00031DDE298B010130E6000130E700203021
:1003AA00E800AA250230E6000130E7002030E80024
:1003BA00AA252C08003A031D052A2B08013A031D19
:1003CA00F429AB01C10A4108653A031DEE296430DC
:1003DA00C1004108E00011260130AD00042A42089C
:1003EA00013A031D042AC201C1034108FF3A031D51
:1003FA00FF29C1014108E00011260130AD00472A5A
:10040A002C08013A031D472A2B08013A031D282A02
:10041A00AB010A304B07F1007108CB007108643A4E
:10042A00031D192ACB01C50A45086D3A031D1F2A67
:10043A006C30C5004508E0004B08E100B7220130E6
:10044A008312A600472A4208013A031D472AC2011D
:10045A000A304B02F1007108CB007108F63A031D0D
:10046A00392A5A30CB00C5034508563A031D3F2A9C
:10047A005730C5004508E0004B08E100B7220130BB
:08048A008312A6000D29482A87
:10049200013083120313E7000030E8008030E900E6
:1004A200EA0169086A0403197F2AE427E427E4279A
:1004B200E427852783160510E427E42783126908B9
:1004C2006605F00000306A05F10070087104031936
:1004D2006D2A83168514702A7A2783168510E427DD
:1004E200E42705148312CA1005187B2ACA1C7A2A2B
:1004F2007B2A752AEA0CE90CEA13522AE701E80181
:10050200E427E427852783160510E427E4278514CA
:10051200E427E427E427E42705148312CA10051808
:10052200962ACA1C952A962A902AE701E801E4270E
:10053200E427851C9D2A6714E427E427E427E4279F
:10054200E427E427E427E427E427E427E427E42751
:10055200E427E427E427E4278527831605107A2772
:0C0562008316851083126708F000080063
:10056E008E3083120313E2006008E6004630E70087
:10057E00DF250130E6000230E7004630E800B62401
:10058E002E30EB00AF276108003A031DD52A30301C
:10059E00EB00AF273030EB00AF27E02A6108E60012
:1005AE004630E700DF254708EB00AF274808EB0091
:1005BE00AF272230E60004274508F0001430F4007F
:1005CE00EB267008E4007108E5000530F4004B08D6
:1005DE00F000272770086407F40065080318013E31
:1005EE00F5007508F2000030F51BFF30F3007208BD
:1005FE00E000F00170087402E100FF30E3001627FE
:10060E00C0308312E60049226008E60049226108E4
:10061E00E60049226208E60049226308E600492204
:04062E00D0260800CA
:1006320083120313FB017308031D77080319702B40
:1006420072087606FA007708F3077E30031C2D2B1A
:10065200F3020318732B302BF302031C762B720860
:10066200F8007108FC007008FD00F817F617031077
:10067200F201F101F0011830A0007D1C4A2B740830
:10068200F00775080318750FF10776080318760F3F
:10069200F207F20CF10CF00CF80CFC0CFD0C031040
:1006A200A00B3E2BF21B5A2BF80DF00DF10DF20DA3
:1006B200F3037B1B701C6C2BF81F6C2BF00A0319C5
:1006C200F10A0319F20A031D6C2BF20CF10CF00C67
:1006D200F30A0319732BFA1FF2130030782B01303F
:1006E200CD27782B02306227782B04306E2700004A
:0206F2000800FE
:1006F4007C18B02BFC18812B7C19CF2B7A2BA001F2
:100704007208031DA12B7108F2007008F10078082B
:10071400F000F801A0157208031DA12B7108F20066
:100724007008F100F001A01120167208031DA12B1E
:100734007108F200F101A01572080319C32B2008F7
:10074400F302031D031CC72B0310F21BB02BF80D7F
:10075400F00DF10DF20DF30BA72BC72B7B1B701CB7
:10076400CB2BF81FCB2BF00A0319F10A0319F20A59
:10077400031DCB2BF20CF10CF00CF30A0319CF2B55
:10078400CB2B0130FC00CD27D22B0230FC006E278E
:10079400D22B0430FC00E027D22B0830FC00622767
:0407A4000000080049
:1007A800803083120313E2000030E300E401E50126
:1007B800620863040319FF2BE427E42783168514D2
:1007C800E427E42705148312CA100518EF2BCA1C66
:1007D800EE2BEF2BE92B851CF52B6208E40463084C
:1007E800E504E427E4278527831605108312E30C24
:1007F800E20CE313DC2B83168514E427E427831229
:100808006008610403190B2C7A2783168510831658
:10081800E427E42705148312CA100518172CCA1CEC
:10082800162C172C112CE427E4278527831605108E
:10083800E427E4277A278316851083126408F000DA
:020848000800A6
:10084A0083160313851305130612861206138613DD
:10085A008312851305138613061386120612A6271A
:10086A00A627A627861606168517E4278513A62720
:10087A008517E4278513A6278517E4278513A62756
:10088A0006128517E4278513A6278517E4278513FB
:10089A00861286178517E4278513A6278613061658
:1008AA008517E427851306128517E4278513A627DB
:1008BA008517E427851306168517E4278513A627C7
:1008CA0006128517E4278513861706178616061655
:0C08DA008517E4278513A6274A140800A0
:1008E60083120313FB01FC01FA0173080319A02C00
:1008F600FA13F2178630F302F31B842C0319842CA7
:10090600A22CF309F30A08307302031C912CF3009E
:10091600F20DF2017308031D0310982C73080319D6
:10092600982C0310F20CF30B942C7B1B721CA02C3E
:10093600031CA02CF20A0319A72CF101AA2C7B1484
:10094600FB1FAD2CF101AD2C0130FC00AF2C0030AB
:10095600FC00AF2CFF30FC00FC080319B32C482721
:060966007208F000080019
:10096C00C82C803083120313E600DB2CC030E60069
:10097C00DB2C9430E600DB2CD430E600DB2C803012
:10098C00E600DB2C831203136608013A0319B72C1B
:10099C006608023A0319BC2C6608033A0319BF2CEB
:1009AC006608043A0319C22CC52C6703F0006608CC
:1009BC00F0077008E6007008EC00F6244A10E90114
:1009CC0069086807840000080319F42C6908680793
:1009DC0084000008EB00AF27E90AE62C4A14080053
:1009EC0083120313EC1BFC2C8613FD2C86176C1B3B
:1009FC00012D0613022D0617EC1A062D8612072D53
:100A0C0086166C1A0B2D06120C2D06164A18102D74
:100A1C000517112D05138517E4278513EC19182DCF
:100A2C008613192D86176C191D2D06131E2D0617EE
:100A3C00EC18222D8612232D86166C18272D0612E3
:100A4C00282D06164A182C2D05172D2D0513851744
:100A5C00E42785134A1C342DA627352DD4270800EE
:100A6C00831603131208013EF000F1010318F10A7A
:100A7C0083126608F400F50140260630F200700877
:100A8C00F4007108F50072080319512DF50CF40CE3
:100A9C00F513FF3E4A2D0430F1007408F000710884
:100AAC0003195C2DF00D7010FF3E562D83120313AD
:100ABC0030307005F3007408F0007508F100F10C8B
:100ACC00F00CF113F10CF00CF113700895000F30D1
:080ADC00970573089704080058
:100AE40083120313E4016108F1000130F00071087E
:100AF4000319802DF00D7010FF3E7A2D7008E5006B
:100B0400600884000008F00570080130031D0030FF
:100B1400F0006308F0060319A72D6208003C0318CF
:100B2400972DBF27BF27E2038F2D60088400650837
:100B34000005F00070080130031D0030F000630868
:100B4400F0060319A72DFF30E4006408F000080044
:100B5400BC2D803083120313E600CF2DC030E60095
:100B6400CF2D9430E600CF2DD430E600CF2D803049
:100B7400E600CF2D831203136608013A0319AB2D47
:100B84006608023A0319B02D6608033A0319B32D17
:100B94006608043A0319B62DB92D6703F0006608F8
:100BA400F0077008E6004A147008EC00F6244A10B6
:0A0BB4006808EC00F6244A1408005B
:100BBE0083120313E801033068020318ED2D680851
:100BCE006707840020308000E80AE22D6808670776
:100BDE0084008001E80368086707E9000A30F40022
:100BEE006608F00027277808F0003030F007690813
:100BFE008400700880000A30F4006608F000272791
:100C0E007008E6007008003A031D0E2E102EE80341
:040C1E00F22D0800AB
:100C22000D30FC00FB30FD00FD0B152EFC0B152ECC
:100C320000000000023083120313E6000330E700D5
:100C42003330E800B6246008F00038270030F400A2
:100C52000030F5002030F6008030F70019237324AD
:100C62007008E60036256008E6004630E700DF251A
:0E0C72004630E60004272530EB00AF270800CF
:100C800083120313FB01FA01F9018030F800F10C23
:100C9000F00C031C542E7408F90775080318750F1F
:100CA000FA070318FB0A0310F01F5C2E7408FA07FA
:100CB00075080318750FFB07FB0CFA0CF90CF80C00
:100CC000031C472E7B08F3007A08F2007908F10034
:060CD0007808F0000800A6
:100CD600403083120313EC00F624E2016208073C5D
:100CE600031C872E6208E63EF00007300318013E1B
:100CF600F1007008C3007108C400C6278A110A12E1
:100D0600EB00AF27E20A712E0230EC00F6246008F1
:0C0D1600E6006108E700E801AA250800DB
:100D2200FF00030E8301CD000A08CC008A0170087F
:100D3200A1008B1CA82E061CA72E861CA42E0130F7
:100D4200C200AB01A72E0130AB00C2018B102108FB
:100D5200F0004C088A004D0E8300FF0E7F0E090042
:100D6200831603139C1CB72E0000B12E8312600859
:100D720083169B008312610883169A009C131C152C
:100D82000B08F0008B1355309D00AA309D009C1477
:0E0D9200F01BCD2E8B13CE2E8B171C110800DC
:100DA0007A2783168510E427E42705148312CA10D6
:100DB0000518DE2ECA1CDD2EDE2ED82EE427E427F1
:100DC000E427E427E427E427E427E42783168514AF
:060DD000E427E4270800FF
:100DD600831203137008F100F0010830FC0071085B
:100DE600F40C0318FA2EFC0BF32EF1010034031059
:100DF600FF2EF40C0318F107F10CF00CFC0BFC2E83
:020E06000800E2
:100E080083120313E70167086607840000080319C3
:100E1800152F6708660784000008EB00AF27E70A6C
:040E2800072F080088
:100E2C00831603138514E427E4270514E427E42729
:100E3C007A2783168510E427E42785278316051067
:020E4C0008009C
:100E4E0083120313F8010830FC00700DF80D7408BE
:100E5E00F8020318342FF8070310F00DFC0B2C2F9B
:020E6E0008007A
:100E7000831203137008F800FB01FC019E30F3009D
:100E8000FA01F201F101F0010230FC007A230800BE
:100E90007B14FB1F532FF201FA1FFF30F200F10009
:0A0EA000F000FA0DF20CFF3008001C
:100EAA0083160313051485148312CA100518612FBB
:0A0EBA00CA1C602F612F5B2F080097
:100EC400FB14FB1F6C2FFF30F300F200F100F00065
:080ED400FA0DF20CFF300800DA
:100EDC007B15FB1F782F0130F300F201F101F001BB
:080EEC00FA0DF20CFF300800C2
:100EF400053084000008000883120313F000F0108A
:060F0400700880000800E7
:100F0A00053084000008000883120313F0007010F3
:060F1A00700880000800D1
:100F2000C6278A110A128000840AC30A0319C40A58
:080F3000F003031D902F0800DF
:100F380083120313600883169B009C131C141A0861
:040F4800F0000800AD
:100F4C000830FC002330FD00FD0BAA2FFC0BAA2F50
:020F5C0008008B
:100F5E00831203134A106B08EC00F6244A1408009F
:100F6E00831603138611831212150C309704080092
:0E0F7E00A530FD00FD0BC12F00000000080093
:0E0F8C008312031344088A0043088200080001
:0E0F9A00F201F101F001F801F301003008004E
:0C0FA8001030FD00FD0BD62F00000800EB
:0C0FB40083120313950117129712080016
:080FC000FA1FF21300300800D3
:040FC800000008001D
:100FCC000434023401341F341F3401340234043429
:02400E0070211F
:00000001FF
